:030000000239942E
:0C39940078FFE4F6D8FD7581670239DB8E
:101F47000A53746172743A20004950436F6E6E658C
:101F570063745245510A00444843502D4F4B0A00C1
:101F67004950436F6E6E65637400C0E4E0EFF2E5BD
:101F7700F020D1E8EDEAEEEC4950285243290A0057
:101F8700C2E5F0F1E8FF20495020ECEEE4F3EBFF67
:101F97003A20322E3420EEF22032302E31312E32DA
:101FA7003030350A00C4E0F2E020F1EEE7E4E0ED7E
:101FB700E8FF3A2000536570203236203230303641
:101FC70000200031313A32323A3338000A000A50E1
:101FD700524F473A20202020202020202020202058
:101FE70020202020202020202020202020202020EA
:101FF70020202020202020202020202020202020DA
:1020070020202020202020202020202020202020C9
:102017002020202020202020200A0044756D7058A1
:102027002020202020303020303120303220303323
:1020370020303420303520303620303720303820DB
:102047003039203041203042203043203044203086
:10205700452030460A003A200044756D7044202020
:1020670020202030302030312030322030332030D3
:102077003420303520303620303720303820303982
:10208700203041203042203043203044203045204A
:1020970030460A00457272206B65790052642065EC
:1020A7006570726F6D0A005264204D454D0A0044F9
:1020B700656275674950204F4E0A0044656275672F
:1020C7004950204F46460A00446562756755736557
:1020D70072204F6E0A0044656275675573657220FA
:1020E7004F46460A0044656275674D7367204F6E19
:1020F7000A0044656275674D7367204F46460A00BC
:10210700436F6E666967206C6F636B210A005772B5
:1021170020656570726F6D0A0020536176652065D2
:102127006570726F6D210A00457272204D4143211F
:10213700004C6F61643E3E00576169745265737469
:1021470061727421004E4F4950004C494E4B434F2A
:102157004E5452005452415353004652004E4F4C76
:10216700494E4B00494E490000FF214CFF2151FFCA
:0E217700215BFF2161FF2164FF216BFF216FBF
:0641E000010B00010900C3
:10415A00C2AFC28E758900438910758BFF758DB702
:07416A00D2ABD28ED2AF22CE
:03001B0002386F39
:10386F00C0E0C083C082C0D0C2AFC28E758BFF755F
:10387F008DB720170675A61E75A6E10509D213E5AB
:10388F000B6002050B050EE50E540F7053D21EE5AB
:10389F000E543F7014D211907A83E0600C04F0E064
:1038AF00D394B44004C2AF80FE907A7EE0600204ED
:1038BF00F0E50AD394014002150A90757BE060028F
:1038CF0014F0907A84E0D394014003E014F03016A2
:1038DF0002050CE50DD394644004D2178002050D48
:1038EF00E508D3940140021508D28ED2AFD0D0D0C4
:0638FF0082D083D0E0320C
:103F0900E4FFFEFD74512DF582E43477F583E02F4B
:103F1900FFE43EFE0DBD10ECE4FD74A62DF582E430
:103F29003475F583E0FC2FFFE43EFEEC60040DBD23
:023F390080E81E
:013F3B002263
:10077600C21B7D027C007F071241218F55E555641F
:100786006060097D017F60124074D21BE4FDFC7F2E
:100796000B1241218F55E55530E6097D04E4FF1221
:1007A6004098D21B7D017C007F071241218F55E5C1
:1007B600557008FD7FFF124074D21B301B03126078
:1007C60000C2AFC288D2A8C2AA123905D2AF123F60
:1007D600091225B9123444C217123DD290774FE060
:1007E600C3940350037403F0D21DD21CD21BD293C0
:1007F600201B077E1F7F47122FF5E490796FF012BA
:10080600415AC2AF750A01A3F0C218C219D2AF7518
:10081600A70775A61E75A6E112413E201B19AF5506
:100826007E007D031230DAE4FF1235EE7E777F6FAD
:10083600E4FB7D01123296907A83E060037401F046
:10084600E490757BF0A37455F0A37481F0E4F50C85
:10085600E4F50D90757BE07003122185907A84E0B3
:10086600B401119080007410F0E4907A84F0D21BE9
:10087600D21CD21DE50CD39403402D908002E4F0E7
:10088600908001F0908000F0E50CD394054003744D
:1008960001F0E50CD3940A400FE4F50CC2149079EC
:1008A60070F0750A01123DD29080A0E070077FCBF0
:1008B6007E03123BAF9080B8E0700312369C9080A6
:1008C600D0E07014301F11907A7A74FFF09077435D
:1008D600E0FEA3E0FF123CAF908000E070133018FA
:1008E60010122EE990772BEFF0D394004003120EEE
:1008F6006C908002E07006908000E06005D21602DF
:100906000856C216E4F50C90757BE06003020856A3
:10091600301A15122C6D90772BEFF0D39400400807
:10092600301205E0FF124197201903020B35122AF7
:10093600F090772BEFF07003020856907A83E06010
:10094600037401F090776FE054BF247F7003020AAE
:10095600091470030209EA24026003020AE0201B5C
:10096600077E1F7F50122FF5907747E0FF700690A5
:10097600774BE06055907A7AE0FEB50722A3E0FF58
:10098600907748E0B50718907A7CE0FF907749E0C9
:10099600B5070C907A7DE0FF90774AE06F602B9068
:1009A600774BE06E7035907A7BE0FF90774CE0B540
:1009B6000729907A7CE0FF90774DE0B5071D907A85
:1009C6007DE0FF90774EE0B50711C2149079707400
:1009D60003F0120021750A01020B35907A7A74FF32
:1009E600F0020B35907A72E0FF907771E06F60034A
:1009F600020B35907A72E004F0E4F50A90796FF014
:100A0600020B35301403020B35907770E0D3940A4D
:100A16005003020AB3A3E064026003020AB39077AC
:100A260038E0FF90777AE06F6003020856907739D6
:100A3600E0FF90777BE06F600302085690773AE01C
:100A4600FF90777CE06F600302085690773BE0FFEB
:100A560090777DE06F600302085690773CE0FF9048
:100A6600777EE06F600302085690773DE0FF90774F
:100A76007FE06F60030208567E1F7F5E122FF5909F
:100A8600777263A20190773063A2017F12122875F4
:100A960090778463A201907A7A63A2017F04122878
:100AA600759079707406F0750A02020856743E4411
:100AB6007770030208561241F5D214E4F50A9079CC
:100AC6006FF0907A7E04F0E4907A71F0A3F0201B28
:100AD6005E7E1F7F67122FF5805530145290776F18
:100AE600E020E74B907771E0FF907A71E0FE6F604F
:100AF6000D907A79E07007EE146F70338013907A58
:100B060071E004F090772BE0FFD394044003123E8B
:100B1600D59074777482F0A37401F0907771E090A9
:100B26007479F07E747F777D03123C30020856207C
:100B36001403020BF19080D0E0700B907743E0FE37
:100B4600A3E0FF123CAFE50A7066907A7EE0D3948C
:100B56003C4037907A79E07031120006907A7E74C4
:100B660001F0E490786FF0A37412F0907A72E0903E
:100B76007871F0A374FDF090757E63A2019078738E
:100B860063A2017F121228758006123F3CEF602097
:100B96007E787F6F907870E02404FD123C30907A66
:100BA60079E0600302085690774FE0F50A0208568E
:100BB6001241CDEF60159074777483F0E4A3F07E54
:100BC600747F777D02123C30020856E50A640160A4
:100BD6000302085690796FE004F0E0C3940540B034
:100BE600C214E4A3F0120021020856E50A6401606B
:100BF60003020856907970E0147003020C95147085
:100C060003020CC1147003020D69147003020E1F57
:100C160024FE606924066003020856E4F50CF555C7
:100C260074272555F582E43476F583E0FF74302584
:100C360055F582E43477F583EFF00555E555B43F75
:100C4600DF201F2190774763A201907A7A63A20181
:100C56007F041228759079707401F090796FF075A1
:100C66000A030208569079707404F090796F740143
:100C7600F0750A14907A7A74FFF0020856E4F50CBF
:100C8600123DD29079707401F0750A0302085690ED
:100C96007A7AE0600B907743E0FEA3E0FF123CAF68
:100CA600750A029079707402F090773EE070030244
:100CB60008569079707403F0020856907A7AE070BC
:100CC60003020D5A90786F7480F09078717402F078
:100CD600E4A3F0A304F090773863A20190787463DC
:100CE600A2017F0A12287590787E7430F0A3747B77
:100CF600F0E4F55574A62555F582E43475F583E0E0
:100D0600FF601174802555F582E43478F583EFF0A1
:100D1600055580E074802555F582E43478F58374B2
:100D26007DF074812555F582E43478F583E4F0E5A9
:100D3600552411907870F07C7A7D7A907743E0FAAA
:100D4600A3E0FB7F02123B2B7E787F6FE5552413D1
:100D5600FD123C309079707404F090774FE0F50AFC
:100D6600020856907A7AE07003020E1090786F743B
:100D760080F09078717401F0E4A3F0A304F0A374FA
:100D860030F0A3747BF0E4F55574A62555F582E49E
:100D96003475F583E0FF601174762555F582E434E9
:100DA60078F583EFF0055580E074762555F582E4F5
:100DB6003478F583747DF074772555F582E43478BC
:100DC600F583E4F0E5552407907870F07C7A7D7A17
:100DD600907743E0FAA3E0FB7F02123B2B7E787FFD
:100DE6006FE5552409FD123C30907A79E0601B12BC
:100DF60041F5D214E4F50A90796FF0907A7E04F00A
:100E0600E4907A71F0A3F00208569079707404F0B9
:100E160090774FE0F50A020856907A7AE0FF60096B
:100E2600F460069080027410F0201F2B750A029061
:100E3600796FE06401FFF0A37401F0EF600590772D
:100E460047800390774B63A201907A7A63A2017F71
:100E560004122875020856750A14907A7A74FFF0FF
:050E660002085680FEA9
:010E6B002264
:100E6C00907770E0B444047F0180027F0090776F2C
:100E7C00E0B447047E0180027E00EE5F604A90770A
:100E8C0038E0907771F0907739E0907772F0907746
:100E9C003AE0907773F090773BE0907774F090772E
:100EAC003CE0907775F090773DE0907776F0907716
:100EBC00707452F090772563A2019080A863A20110
:100ECC007F0612287502137A90772BE0C394085092
:100EDC0003021383907738E0FF907771E06F600323
:100EEC00021383907739E0FF907772E06F60030212
:100EFC00138390773AE0FF907773E06F60030213EF
:100F0C008390773BE0FF907774E06F60030213836C
:100F1C0090773CE0FF907775E06F6003021383904D
:100F2C00773DE0FF907776E06F6003021383907A51
:100F3C0083E060037401F0907A847464F0907770AD
:100F4C007452F090776FE0644D703C7E1F7F71128D
:100F5C002FF57E1F7F87122FF51241D87E1F7FAC95
:100F6C00122FF57E1F7FBC122FF57E1F7FC8122F0C
:100F7C00F57E1F7FCA122FF57E1F7FD3122FF57EB1
:100F8C001F7FD5122FF52290776FE0644C70527E44
:100F9C00207F22122FF5907777E0F556A3E0F557D6
:100FAC00E4F5587D03AF57AE561230DA7E207F5DE4
:100FBC00122FF5AE56AF57E4FB7D101232967E1F02
:100FCC007FD3122FF574102557F557E43556F55687
:100FDC000558E558C3941040CA7E1F7FD3122FF5D5
:100FEC002290776FE0646C705CF55A7E207F601203
:100FFC002FF5E4F559AF5A7E007D031230DA7E20CE
:10100C007F5D122FF5E4F558A85AE6FF7479255840
:10101C00F582E43477F583EFF0055A0558E558B4BA
:10102C0010E67E777F79E4FB7D101232967E1F7F6F
:10103C00D3122FF50559E559C3940840B87E1F7F8C
:10104C00D3122FF52290776FE0644B7046F55874ED
:10105C00612558F582E43477F583E0FF60167477E8
:10106C002558F582E43477F583E0B507100558E58B
:10107C0058B408DB90757B7432F002137A90776F5A
:10108C007421F0301B0302137A7E207F9B122FF504
:10109C0002137A90776FE06452704E201B077E200B
:1010AC007FA3122FF5907778E090772BF0E4F5582A
:1010BC0090772BE0FDE558C39D5022907777E02583
:1010CC00582426F582E43476F583E0FF74792558AC
:1010DC00F582E43477F583EFF0055880D37E777F83
:1010EC006FED240AFD123A202290776FE06449706C
:1010FC0045201B077E207FAE122FF5907777E0F509
:10110C0056A3E0F557E4F558855782855683E0FFE2
:10111C0074792558F582E43477F583EFF00557E5BB
:10112C0057700205560558E558B480DC7E777F6F02
:10113C007D8A123A202290776FE06444600302119A
:10114C00D3907777E0FF6444700302137AEFB431E5
:10115C000CC21B7E207FB6122FF502137A90777784
:10116C00E0B4300CD21B7E207FC2122FF502137A12
:10117C00907777E0B4320CD21C7E207FCF122FF503
:10118C0002137A907777E0B4330CC21C7E207FDD9B
:10119C00122FF502137A907777E0B4340CD21D7EBF
:1011AC00207FEC122FF502137A907777E0B4350C90
:1011BC00C21D7E207FF9122FF502137A907777E00B
:1011CC00FF12001E02137A90757BE07013201B0730
:1011DC007E217F07122FF590776F7421F002137A1E
:1011EC0090757B7432F090776FE0FFB45104C2AF0E
:1011FC0080FEEF64577045201B077E217F15122F50
:10120C00F5907778E090772BF0E4F55890772BE019
:10121C00FFE558C39F400302137A74792558F58271
:10122C00E43477F583E0FF907777E025582426F5B2
:10123C0082E43476F583EFF0055880D090776FE038
:10124C00645360030212F5201B077E217F20122FAE
:10125C00F5907738E0FF90762FE06F703C907739FF
:10126C00E0FF907630E06F703090773AE0FF907648
:10127C0031E0B5072490773BE0FF907632E0B5077C
:10128C001890773CE0FF907633E0B5070C90773DF3
:10129C00E0FF907634E06F601690776F7421F03039
:1012AC001B0302137A7E217F2F122FF502137AE48F
:1012BC00F558E4F50D74262558F582E43476F5835B
:1012CC00E0FDAF58123FCD0558E558C394FE40E2FF
:1012DC00C2AFE4907FF0F0A3F0907FFD74AAF0A36E
:1012EC0074FFF0A37455F080FE90776FE0644F703C
:1012FC004B907777E0F556A3E0F557E557455670D8
:10130C000A201B077E217F38122FF5201B077F2A0E
:10131C007E00122FF5E4F55874792558F582E434E3
:10132C0077F583E0855782855683F00557E557702E
:10133C000205560558E558B480DE803290776FE090
:10134C00B4452B201B077E217F3F122FF59077771A
:10135C00E0FFA3E0907FF0CFF0A3EFF0C2AF907F5F
:10136C00FD74AAF0A374FFF0A37455F080FE7E7791
:07137C007F6F7D08123A208B
:011383002247
:103E9D00AE07EEC39430400BEED394395005EE24AB
:103EAD00D0FF22EEC39461400BEED394665005EE25
:103EBD0024A9FF22EEC39441400BEED39446500546
:083ECD00EE24C9FF22AF06221A
:1025B900C212E4907A83F0D21FC215907A79F09012
:1025C900773863A201907A7363A2017F0612287596
:1025D900E4F556E55675F003A42470F582E4342138
:1025E900F583E493FB740193FA740293F9121C17AF
:1025F9007003022799E4F557F558FD74A62DF58265
:10260900E43475F583E0FF7003022794E55675F00D
:1026190003A42470F582E43421F583E493FB740167
:1026290093FA740293F9855782758300121C30FE60
:10263900EFB506087558010557022790E55870034C
:10264900022790EE600302278BE55624FE602214D0
:10265900700302277B14700302277F14700302277B
:102669008724046003022794907A837401F0022777
:1026790094D21274A62DF582E43475F583E0FF64D3
:102689002D7003022794123E9DEFC454F0FC74A7E9
:102699002DF582E43475F583E0FF123E9DEF2C9011
:1026A9007A73F074A82DF582E43475F583E0FF128E
:1026B9003E9DEFC454F0FC74A92DF582E43475F500
:1026C90083E0FF123E9DEF2C907A74F074AA2DF5E9
:1026D90082E43475F583E0FF123E9DEFC454F0FCAB
:1026E90074AB2DF582E43475F583E0FF123E9DEF5E
:1026F9002C907A75F074AC2DF582E43475F583E08D
:10270900FF123E9DEFC454F0FC74AD2DF582E43404
:1027190075F583E0FF123E9DEF2C907A76F074AE4A
:102729002DF582E43475F583E0FF123E9DEFC45424
:10273900F0FC74AF2DF582E43475F583E0FF123EA9
:102749009DEF2C907A77F074B02DF582E43475F50D
:1027590083E0FF123E9DEFC454F0FC74B12DF58265
:10276900E43475F583E0FF123E9DEF2C907A78F002
:102779008019D2158015907A797401F0800DC21FE5
:102789008009E4F558F5570D02260405560225DCA3
:01279900221D
:03000300023D16A5
:0D3D1600C0E0C083C082C0D075D000C007DF
:103D2300C2A8908008E0FFEF54F06035EF30E4085C
:103D3300D2189080087410F0EF30E508D21A908002
:103D4300087420F0EF30E608D2199080087440F030
:103D5300EF30E7069080087480F0908008E0FF80E1
:093D6300C690800874FFF0D2A89C
:0B3D6C00D007D0D0D082D083D0E0324E
:103DD2009080007480F090773063A201F583F582C1
:103DE20063A2017F0812287590773863A201908040
:103DF2008863A2017F0A122875907742E0FF9080C3
:103E0200B1F09080E1EFF09080957455F0A3F090BE
:0C3E120080007401F09080097470F022B0
:043BAF00AD07AC06AC
:103BB300908009E04410F09080A0E0706F9080A1A5
:103BC3007482F09080A874FFF0A3F0A3F0A3F0AF89
:103BD30004AE079080AEEEF0AE05A3EEF0AE079014
:103BE30080ACEEF0AE05A3EEF09080007402F0908E
:103BF3007BA3121D6C00000000907BA3E09080402B
:103C0300F0907BA4E0908041F0907BA5E09080420F
:103C1300F0907BA6E0908043F0A3E4F0A3F0A3F040
:0C3C2300A3F0908018F0A3F0A3F0A3F031
:013C2F002272
:043CAF00AD07AC06AB
:103CB300908009E04440F09080D0E070559080D12E
:103CC3007482F0AF049080DEEFF0AF05A3EFF090C5
:103CD30080027402F0907BA7121D6C00000000901C
:103CE3007BA7E0908058F0907BA8E0908059F090FB
:103CF3007BA9E090805AF0907BAAE090805BF0A3D0
:103D0300E4F0A3F0A3F0A3F0908030F0A3F0A3F0CD
:023D1300A3F01B
:013D1500228B
:10369C00908009E04420F09080B8E0600302373D50
:1036AC009080B97482F07F039080C6EFF07FCDA339
:1036BC00EFF07F039080C4EFF0A374CDF0300022C4
:1036CC00907747E09080C0F0907748E09080C1F010
:1036DC00907749E09080C2F090774AE09080C3F0F8
:1036EC00800C9080C074FFF0A3F0A3F0A3F0908046
:1036FC00017402F0907BAB121D6C00000000907BFB
:10370C00A7E090804CF0907BA8E090804DF0907BEF
:10371C00A9E090804EF0907BAAE090804FF0A3E45B
:10372C00F0A3F0A3F0A3F0908024F0A3F0A3F0A3F7
:01373C00F09C
:01373D002269
:103B2B008C568D57A907EAFDE975F018A424ACFF54
:103B3B00E5F034808F82F583EDF0EBFDE975F0183D
:103B4B00A4FFAEF024ACFBEE34808B82F583A3EDA7
:103B5B00F08557828C83E0FDEF24A8FFEE3480FEC6
:103B6B008F82F583EDF08557828C83A3E08F828E55
:103B7B0083A3F0855782855683A3A3E0FDE975F0F7
:103B8B0018A424A8FFE5F03480FE8F82F583A3A34D
:103B9B00EDF08557828C83A3A3A3E08F828E83A342
:043BAB00A3A3F022BE
:063A20008D5BAB07AA0656
:103A2600907BA3E0FCA3E0FDA3E0FEA3E0F55F8EA0
:103A36005E8D5D8C5CAE02AF038E838F8263A201C6
:103A4600E55E540744C0F583855F8263A201AF5BE0
:103A56001228DE908000E020E5F9E4FCFDFEE55F3B
:103A6600255BF55FEE355EF55EED355DF55DEC35B6
:103A76005CF55CC2A8908040E55CF0A3E55DF0A330
:103A8600E55EF0A3E55FF0D2A89080007420F0AF69
:0F3A96005FAE5EAD5DAC5C907BA3121D60AF5B5D
:013AA50022FE
:063C30008D56AB07AA0649
:103C3600907BA7E0FCA3E0FDA3E0FEA3E0F55A8E8F
:103C4600598D588C57AE02AF038E838F8263A201C3
:103C5600E559540744D0F583855A8263A201AF56CD
:103C66001228DEE4FCFDFEE55A2556F55AEE3559D6
:103C7600F559ED3558F558EC3557F557C2A89080EB
:103C860058E557F0A3E558F0A3E559F0A3E55AF037
:103C9600D2A89080027420F0AF5AAE59AD58AC57F6
:083CA600907BA7121D60AF56D0
:013CAE0022F3
:0235EE008F57F5
:1035F000908001E030E5037F0022907BABE0FCA3EC
:10360000E0FDA3E0FEA3E0F55B8E5A8D598C589047
:103610007A7363A201E55A540744C8F583855B8237
:1036200063A2017F061228F4E55B2406F55BE4350E
:103630005AF55AE43559F559E43558F558907971E9
:1036400063A201E55A540744C8F583855B8263A2EF
:1036500001AF571228F4E4FCFDFEE55B2557F55B4E
:10366000EE355AF55AED3559F559EC3558F558C23D
:10367000A890804CE558F0A3E559F0A3E55AF0A3D3
:10368000E55BF0D2A89080017420F0AF5BAE5AAD3C
:0B36900059AC58907BAB121D60AF5787
:01369B00220C
:102EE900C2A89081E0E0F5560556055605560556E7
:102EF900055605560556055605560556908010E0A7
:102F0900F559A3E0F55AA3E0F55BA3E0F55C9081E0
:102F1900E1E0F5560556055605560556055605567A
:102F29000556055605560556908014E0F55DA3E053
:102F3900F55EA3E0F55FA3E0F560D2A8E55FB55BB8
:102F490008E560B55C037F0022E4F556E55F5407A8
:102F590044E0F58385608263A20190776F63A201E3
:102F69007F0812290C90777163A20190772563A2DB
:102F7900017F0612287590776FE0F557A3E0F558A1
:102F8900E4F55690776FE0702AA3E024F8F556E54A
:102F99005F540744E0F58385608274082582F582D1
:102FA900E43583F58363A20190776F63A201AF567D
:102FB90012290CAE57E4FCFDE5602558F560E55F84
:102FC9003EF55FED355EF55EEC355DF55DC2A890C9
:102FD9008014E55DF0A3E55EF0A3E55FF0A3E5608D
:0B2FE900F0D2A89080007440F0AF56BA
:012FF40022BA
:102AF000C2A89081E6E0F5560556055605560556DE
:102B0000055605560556055605560556908028E08B
:102B1000F559A3E0F55AA3E0F55BA3E0F55C9081DD
:102B2000E7E0F55605560556055605560556055671
:102B3000055605560556055690802CE0F55DA3E038
:102B4000F55EA3E0F55FA3E0F560D2A8E4F556E5F5
:102B50005FB55B0AE560B55C05C219022C4EE55F06
:102B6000540744F0F58385608263A20190776F6318
:102B7000A2017F0812290C90776FE0F557A3E0F5CA
:102B800058E558455770099080027410F07F002274
:102B9000907A7AE0FFF4602D907771E06F70769014
:102BA0007A7BE0FF907772E06F706A907A7CE0FF4A
:102BB000907773E06F705E907A7DE0FF907774E0BD
:102BC0006F60228050907771E0907A7AF0907772FF
:102BD000E0907A7BF0907773E0907A7CF090777455
:102BE000E0907A7DF090776FE0702AA3E024F8F50A
:102BF00056E55F540744F0F58385608274082582AA
:102C0000F582E43583F58363A20190776F63A201B7
:102C1000AF5612290CAE57E4FCFDE5602558F5606F
:102C2000E55F3EF55FED355EF55EEC355DF55DAF7C
:102C30005CAE5BAD5AAC59AB60AA5FA95EA85DD330
:102C4000121D4F40099080027410F07F0022C2A82C
:102C500090802CE55DF0A3E55EF0A3E55FF0A3E5D1
:0C2C600060F0D2A89080027440F0AF56E3
:012C6C002245
:102C6D00C2A89081E3E0F556055605560556055662
:102C7D0005560556055605560556055690801CE019
:102C8D00F559A3E0F55AA3E0F55BA3E0F55C90815F
:102C9D00E4E0F556055605560556055605560556F6
:102CAD000556055605560556908020E0F55DA3E0C6
:102CBD00F55EA3E0F55FA3E0F560D2A8E4F556E577
:102CCD005FB55B0AE560B55C05C21A022DB5E55F1F
:102CDD00540744E8F58385608263A20190747B6399
:102CED00A2017F0E12292290747BE0F557A3E0F527
:102CFD0058907A73E0FF907483E06F706C907A74E3
:102D0D00E0FF907484E06F7060907A75E0FF9074CE
:102D1D0085E06F7054907A76E0FF907486E06F7066
:102D2D0048907A77E0FF907487E06F703C907A78E6
:102D3D00E0FF907488E06F703090747BE0702AA390
:102D4D00E024F2F556E55F540744E8F5838560828B
:102D5D00740E2582F582E43583F58363A2019074A8
:102D6D007B63A201AF56122922AE57E4FCFDE5604C
:102D7D002558F560E55F3EF55FED355EF55EEC35AA
:102D8D005DF55DAF5CAE5BAD5AAC59AB60AA5FA9AA
:102D9D005EA85DD3121D4F5006E55845577009903A
:102DAD0080017410F07F0022C2A8908020E55DF0B4
:102DBD00A3E55EF0A3E55FF0A3E560F0D2A89080F7
:062DCD00017440F0AF5656
:012DD30022DD
:042FF5008E5B8F5C04
:102FF900907BA3E0FCA3E0FDA3E0FEA3E0F5628ED5
:10300900618D608C5FE562FFE5615407FEE42FF591
:103019005EEE34C0F55D855E82F5837423F0055E4E
:10302900E55E7002055D535DC7F582855D83740AAF
:10303900F0055EE55E7002055D535DC79077386304
:10304900A201855D83855E8263A2017F061228DE67
:103059007406255EF55EE4355DF55D855B83855C0B
:103069008263A201855D83855E8263A2011228C203
:10307900908000E020E5F9E4FCFDFE907BA3E0F8F8
:10308900A3E0F9A3E0FAA3E02FFFEE3AFEED39FD44
:10309900EC38FCEF2408FFE43EFEE43DFDE43CFC93
:1030A900907BA3121D60C2A8907BA3E0908040F0A2
:1030B900907BA4E0908041F0907BA5E0908042F065
:1030C900907BA6E0908043F0D2A89080007420F015
:0130D90022D4
:063296008E5B8F5C8D5D74
:10329C00907BA3E0FCA3E0FDA3E0FEA3E0F5638E2E
:1032AC00628D618C60E563FFE5625407FEE42FF5E7
:1032BC005FEE34C0F55E855F82F5837423F0055FA5
:1032CC00E55F7002055E535EC7F582855E83EBF0A9
:1032DC00055FE55F7002055E535EC790773863A2A9
:1032EC0001855E83855F8263A2017F061228DE74EE
:1032FC0006255FF55FE4355EF55E855B83855C8254
:10330C0063A201855E83855F8263A201AF5D122893
:10331C00DE908000E020E5F97408255DF55DFFE4A2
:10332C00FCFDFEE5632FF563EE3562F562ED35616C
:10333C00F561EC3560F560C2A8908040E560F0A3C3
:10334C00E561F0A3E562F0A3E563F0D2A8908000FC
:10335C007420F0AF63AE62AD61AC60907BA3121DC4
:01336C006000
:01336D00223D
:0630DA008E5B8F5CAB056C
:1030E000907BA3E0FCA3E0FDA3E0FEA3E0F5628EED
:1030F000618D608C5FE562FFE5615407FEE42FF5AA
:103100005EEE34C0F55D855E82F5837423F0055E66
:10311000E55E7002055D535DC7F582855D83EBF06A
:10312000055EE55E7002055D90773863A201855DFE
:1031300083855E8263A2017F061228DE7406255E07
:10314000F55EE4355DF55D535DC7E55B855E8285C3
:103150005D83F0055EE55E7002055D535DC7F58237
:10316000855D83E55CF0055EE55E7002055D535D9F
:10317000C7908000E020E5F9E562240AF562E435B5
:1031800061F561E43560F560E4355FF55FC2A890F4
:103190008040E55FF0A3E560F0A3E561F0A3E562A0
:1031A000F0D2A89080007420F0AF62AE61AD60AC48
:0731B0005F907BA3121D607C
:0131B70022F5
:10390500E4F556E55604FF123FF774302556F58267
:10391500E43477F583EFF00556E556C3943F40E36D
:10392500E4F556E556247FFF123FF774A62556F5B4
:1039350082E43475F583EFF074A62556F582E434F8
:1039450075F583E0701D74A62556F582E43475F58A
:10395500837420F074A72556F582E43475F583E465
:10396500F080090556E556C3948040B7E490762566
:10397500F0F556AF56123FF774262556F582E43416
:0E39850076F583EFF00556E556C394FE40E557
:013993002211
:10410100E4FDFCC3ED9FEC9E5015E4FBFA0BBB00F4
:0F411100010ABA01F8BB90F50DBD00010C80E466
:01412000227C
:0D41A6004390014390025390FE5390FD2280
:0D41B3005390FD5390FE4390024390012273
:0E4188005390FD439002E5905408FF5390FDC4
:014196002206
:0D41C0005390FD4390014390025390FD2267
:0741E700AE071FEE70FA2283
:023FA100AD076A
:103FA300E4FC5390FDEDA804088002C333D8FC3031
:103FB300E70543900180035390FE7F051241E743D9
:093FC30090020CBC08DC5390FDD7
:013FCC0022D2
:10404B00E4FF5390FD7E07439002E59030E00D7442
:10405B0001A806088002C333D8FC42075390FD1E0B
:08406B00C3EE6480948050DF75
:01407300222A
:103FCD00AB05AA071241A67FA0123FA1124188AFEF
:103FDD0002123FA1124188AF03123FA11241881274
:0A3FED0041B37F0A7E001241012259
:023FF700AB0716
:103FF9001241A67FA0123FA1124188AF03123FA12F
:104009001241881241A67FA1123FA1124188124094
:074019004B1241C01241B33C
:01402000227D
:10412100A2AF9225C2AF8C838D82EF12293A43A2AE
:0C4131002012293C53A2DFA22592AFFF10
:01413D00225F
:024074008F5665
:10407600A2AF9225C2AFE4F5838D82740612293A67
:10408600E55643A22012293C53A2DFA22592AF7F18
:014096000128
:014097002206
:024098008F5641
:10409A00A2AF9225C2AFE4F5838D82740A12293A3F
:1040AA00E55643A22012293C53A2DFA22592AF7FF4
:0140BA000104
:0140BB0022E2
:10279A00A907E7FFA805EF93C3966008403B74FCBE
:1027AA002FFF80F00F08EF93C3966008402B74FB4D
:1027BA002FFF80E00F08EF93C3966008401B74FA5E
:1027CA002FFF80D00F08EF93D3966008400B74F95F
:1027DA002FFF80C01F1F1F1F1FEF54FEF80303F7B0
:1027EA00E893FC08E893FD08E893FE08E893FF22C3
:1027FA0009E993C39D6008402974FB29F980F1090E
:10280A00E993C39E6008401A74FA29F980E209E93B
:10281A0093D39F6008400B74F929F980D3191919C9
:10282A001919E9C313C313FF22740093F8ECC39870
:10283A004024701F740193F8EDC398401970147402
:0E284A000293F8EEC398400E7009740393F8E1
:10285800EFC39840037F00227F0122EDF8E6F008DD
:10286800A3DFFA22EDF8E0F608A3DFFA22E0A3637B
:10287800A201F0A363A201DFF475A20022E0A36322
:10288800A201F0A363A201E0A363A201F0A363A2E3
:1028980001E463A201F0A363A201DFE175A20022B3
:1028A800E0A363A2016DFE936CFDEE058393FC1516
:1028B8008363A201DFEA75A200227F00E493A36389
:1028C800A201F00F600CA3E583C2E3F58363A201C4
:1028D80080EA75A20022E0A363A201F0A3E583C207
:1028E800E3F58363A201DFEE75A20022E0A363A2F1
:1028F80001F0A3E583C2E4D2E3F58363A201DFEC30
:1029080075A20022E583C2E3F583E0A363A201F088
:10291800A363A201DFEE75A20022E583C2E4D2E33D
:10292800F583E0A363A201F0A363A201DFEC75A223
:102938000022F922C002C004C00612FFF0D006D05F
:0429480004D0022293
:103E1E0020536572763A0020547261737353656E47
:103E2E00644552520A00205265496E69742043411E
:103E3E004E0A002043414E283029203E20544F2167
:103E4E000A0020545520300A0020545520310A0013
:03001E00E4FF22DA
:103F6F00C28DC2AF438901C28C907A99E0FF70076E
:103F7F00F58A758CEE8016EFB40508E4F58A758C1A
:103F8F00B8800AEFB40A06E4F58A758C70D28CD229
:023F9F00AF224F
:103E5E00C28DC2AF438901C28C907A99E0FF701473
:103E6E00302409F58A758CDCC224801E758A66752D
:103E7E008CFC8016EFB40508E4F58A758CEE800A8A
:0F3E8E00EFB40A06E4F58A758CDCD28CD2AF2231
:10413E0012336E120022D223E4F550907BA1F0F5DB
:0C414E003EF554123F6FC224E4F55222EB
:103ED500EF24FCF556201B127E3E7F1E122FF57E29
:103EE500777F737B01AD5612329690777363A2018B
:103EF500907B2163A201AF5612287585563EE4F5E5
:033F05004FC22187
:013F08002296
:0F419700D3EF6480948E5006E55470028F54224B
:10218500208D03022222C28C202303022285E53EF4
:1021950060547425254FF582E4347BF583E02405EE
:1021A500F556D3940E4008E4F53ED22102228574FB
:1021B50021254FF582E4347BF5837D40AF56122807
:1021C5006CE556254FF54FE54030E702D224123F26
:1021D5006F12351AE54FC3953E5003022285E4F58B
:1021E5003ED221022285E5516015907A857D40FF1A
:1021F50012286C123F6F12351AE4F551022285E55B
:1022050054601490747B7D40FF12286C123F6F124E
:10221500351AE4F5548069123AA6123F6F1237D881
:102225008F56EF605B123E5EE4F552E540547EB595
:102235004003123D77E553C3946E5018749A2553A5
:10224500F582E4347AF583E5562553F5537D40AFA1
:1022550056122863301224E54030E70330001C9005
:1022650079717D40AF56122863AF561235EEEF7087
:102275000A201B077E3E7F25122FF5AF56122DD45F
:10228500301E1230110D0552E552D394F04004C2B0
:10229500AF80FEC21E2013030223A0906001E0045C
:1022A500F07006906000E004F0E5506031D39401D1
:1022B500400415508028907BA1E004F0E0D39403FE
:1022C500400D201B077E3E7F34122FF512413E2024
:1022D5001B077E3E7F41122FF5E4F550D2233022B5
:1022E50043E551703F907A8504F0A37408F0A37418
:1022F50080F0A37401F0A37406F0907B1CE0907A43
:102305008AF0907B1DE0907A8BF0907B1EE0907AAE
:102315008CF0907B1FE0907A8DF0E4A3F0A3F0752C
:10232500510BC222302072907B1AE07035E5517056
:1023350031907A857442F0A37408F0907B1BE0908D
:102345007A87F0907B20E0907A88F0A37401F0758D
:102355005106201B077E3E7F50122FF5907B1AE019
:1023650004F0907B1AE06402702FE551702B907A8F
:10237500857402F0A37408F0907B1BE0907A87F0D7
:10238500A3F0A37401F0755106201B077E3E7F570D
:0E239500122FF5907B1AE004F0C213120026FE
:0123A3002217
:103F3C00E553602CE490786FF0A3E553F0907A721F
:103F4C00E0907871F0A37419F0907A9A63A20190C2
:103F5C00787363A201AF53122875E4F5537F0122E5
:033F6C007F0022B1
:0B41CD00302105C2217F01227F00226B
:0100210022BC
:0641F500E4F553F53E2243
:100006007F01E490757EF0A3F0A3F0FEEF25E0FFFC
:040016000EBE08F81A
:01001A0022C3
:0741EE0020457272210A0056
:10417100EF600A7B10E4FD7F0C124021227B107D51
:07418100107F0C1240212207
:10336E00D29475C353C29475C5C0E5C4B480FB85B1
:10337E00C557D2947DE07F0F1240E0907A99E044D9
:10338E0080FD7F2A1240E07D247F291240E07D04DB
:10339E007F281240E0E4FD7F2B1240E0755920E4B7
:1033AE00F558E4FDAF591240E005590558E558C3EC
:1033BE00940840EEE4F559F558E4FDAF591240E09B
:1033CE0005590558E558C3940C40EE7D087F05124B
:1033DE0040E0755910E4F558E4FDAF591240E00590
:1033EE00590558E558C3940C40EE7D3C7F0C1240B5
:1033FE00E07D077F0F1240E07DFF7F2B1240E075CE
:10340E005930E4F557E4F558E4FDAF591240E005A4
:10341E00590558E558C3940E40EE05590559055700
:10342E00E557C3940340DE7D047F601240E0E4FD67
:05343E007F701240E068
:013443002266
:1040BC00C29475C503E5C4B480FBAEC58FC5E5C419
:1040CC00B480FBAEC5E4F5C5E5C4B480FBAEC5D287
:0340DC0094AF0698
:0140DF0022BE
:1040E000C29475C502E5C4B480FBAEC58FC5E5C4F6
:1040F000B480FBAEC58DC5E5C4B480FBAEC5D2941B
:01410000229C
:10402100C29475C505E5C4B480FBAEC58FC5E5C4B2
:10403100B480FBAEC58BC5E5C4B480FBAEC58DC5F0
:09404100E5C4B480FBAEC5D294C5
:01404A002253
:1031B800C29475C503E5C4B480FBAEC5EF60047E58
:1031C8007080027E608EC5E5C4B480FBAEC5E4F5B0
:1031D800C5E5C4B480FB85C53FE4F5C5E5C4B48046
:1031E800FB85C540E4F5C5E5C4B480FB85C541E46D
:1031F800F5C5E5C4B480FB85C542E4F5C5E5C4B4AE
:1032080080FB85C543E4F5C5E5C4B480FB85C544AA
:10321800E544540FFE60741EE4F5C5E5C4B480FBB4
:1032280085C545EE60651EE4F5C5E5C4B480FB853B
:10323800C546EE60561EE4F5C5E5C4B480FB85C5F9
:1032480047EE60471EE4F5C5E5C4B480FB85C54874
:10325800EE60381EE4F5C5E5C4B480FB85C549EECB
:1032680060291EE4F5C5E5C4B480FB85C54AEE6057
:103278001A1EE4F5C5E5C4B480FB85C54BEE600BAA
:0D328800E4F5C5E5C4B480FB85C54CD294C7
:013295002216
:10351A00C29475C502E5C4B480FBAFC575C531E573
:10352A00C4B480FBAFC5E544540FFE8540C5E5C46D
:10353A00B480FBAFC58541C5E5C4B480FBAFC58582
:10354A0042C5E5C4B480FBAFC58543C5E5C4B480B4
:10355A00FBAFC58544C5E5C4B480FBAFC5EE606C5E
:10356A001E8545C5E5C4B480FBAFC5EE605E1E8509
:10357A0046C5E5C4B480FBAFC5EE60501E8547C59D
:10358A00E5C4B480FBAFC5EE60421E8548C5E5C4FC
:10359A00B480FBAFC5EE60341E8549C5E5C4B4806E
:1035AA00FBAFC5EE60261E854AC5E5C4B480FBAFF5
:1035BA00C5EE60181E854BC5E5C4B480FBAFC5EEE9
:1035CA00600A854CC5E5C4B480FBAFC5D2947F02BE
:1035DA00C29475C581E5C4B480FBAFC5D294755059
:0335EA000AC223EF
:0135ED0022BB
:103D7700C29475C502E5C4B480FBAFC575C541E5FE
:103D8700C4B480FBAFC58540C5E5C4B480FBAFC5EF
:103D97008541C5E5C4B480FBAFC58542C5E5C4B45C
:103DA70080FBAFC58543C5E5C4B480FBAFC5E4F56B
:103DB700C5E5C4B480FBAFC5D2947F02C29475C574
:0A3DC70082E5C4B480FBAFC5D294BE
:013DD10022CF
:103AA600C29475C502E5C4B480FBAFC575C551E5C2
:103AB600C4B480FBAFC57497250FF582E43461F575
:103AC60083E0F5C5E5C4B480FBAFC575C508E5C49C
:103AD600B480FBAFC57498250FF582E43461F58395
:103AE600E0F5C5E5C4B480FBAFC575C50FE5C4B444
:103AF60080FBAFC5050F050F7497250FF582E434DB
:103B060061F583E07002F50FE4F5C5E5C4B480FB0A
:103B1600AFC5D2947F02C29475C584E5C4B480FB58
:043B2600AFC5D294C1
:013B2A002278
:1037D8003092037F00227F2C1240BC8F57E5573070
:1037E800E209D223E4F550907BA1F0E55730E55883
:1037F800201B077E417FEE122FF57F2D1240BC8FD4
:1038080058201B11E557FE7C00E42558FFEC3EFECE
:103818007D031230DAE4FBAD587F2D124021201BC6
:103828001BE55730E016E4FF1231B8E540FE7C0096
:10383800E42544FFEC3EFE7D031230DAAB57E4FD8D
:103848007F2C1240217F0022E4F558E55730E00B29
:10385800E4FF1231B8E5442405F558AB57E4FD7F81
:063868002C124021AF58B4
:01386E002237
:10138400C7E0E3F0F3E7EEF7EDFBE920EEE1F0E090
:10139400E73A20CACF20C8F1E5F2FC207620312EAE
:1013A400303328C8D1C5D2DC290A005452414E5AE0
:1013B400004D415842005254530044454C41590099
:1013C4004E4F4B5654004B5000424F4F5400434134
:1013D4004E004E4557504B54004154004443440082
:1013E40043414E4D4F4E0054454C3A004C434C0043
:1013F4004454420054524300000A4F55543A0044A6
:101404006973636F6E6E6563746564210A004D4F82
:1014140044454D5F4F4B210A004D4F44454D5F43BA
:101424004F4E4E454354210A004D4F44454D5F4CA9
:10143400495354454E210A004D4F44454D5F455292
:10144400524F52210A004D4F44454D5F434F4E4E7B
:101454004543545F4641494C555245210A004D4F7E
:1014640044454D5F444953434F4E4E4543544544D0
:10147400210A005254530A004D6F64656D20696E51
:1014840069740A00CDE5F220EEF2E2E5F2E0210A09
:10149400004469616C696E670A00CEF820E4EBE8E9
:1014A400EDFB210A000ACDE5F220CAE2E8F2E0ED04
:1014B400F6E8E821000A436F6E6620526571210048
:1014C400CCEEE4E5EC20E220F5EE2DF0E5E6E8ECE8
:1014D400E5210A00C1F0E0EAF3E5EC210A000A4341
:1014E4005243204552523A20000A494E3A00436F73
:1014F4006E66205265616479210A00436F6E66202E
:10150400426C6F636B210A00CFF0E8EDFFF2FB2021
:10151400E4E0EDEDFBE520E1E5E720F1EEE5E4E8CC
:10152400EDE5EDE8FF210A000A446174613A200008
:101534003F3F3F0A000089129B24AD36BF48C15A81
:10154400D36CE57EF78108931AA52CB73EC940DB1E
:1015540052ED64FF76028B109926AF34BD4AC3580E
:10156400D16EE77CF5830A9118A72EB53CCB42D9FE
:1015740050EF66FD74048D169F20A932BB4CC55EE6
:10158400D768E17AF3850C971EA128B33ACD44DFDE
:1015940056E960FB72068F149D22AB30B94EC75CCE
:1015A400D56AE378F1870E951CA32AB138CF46DDBE
:1015B40054EB62F97008811A932CA53EB740C952C6
:1015C400DB64ED76FF89009B12AD24BF36C148D39E
:1015D4005AE56CF77E0A8318912EA73CB542CB508E
:1015E400D966EF74FD8B029910AF26BD34C34AD17E
:1015F40058E76EF57C0C851E9728A13AB344CD5666
:10160400DF60E972FB8D049F16A920BB32C54CD75D
:101614005EE168F37A0E871C952AA338B146CF544D
:10162400DD62EB70F98F069D14AB22B930C74ED53D
:101634005CE36AF17800112332465765748C9DAFE0
:10164400BECADBE9F810013322564775649C8DBF8E
:10165400AEDACBF9E82130021367764455ADBC8E7F
:101664009FEBFAC8D93120120377665445BDAC9E6E
:101674008FFBEAD8C94253617004152736CEDFEDDB
:10168400FC8899ABBA5243716014053726DECFFD4E
:10169400EC9889BBAA6372405125340617EFFECC3F
:1016A400DDA9B88A9B7362504135241607FFEEDC2E
:1016B400CDB9A89A8B8495A7B6C2D3E1F008192BAB
:1016C4003A4E5F6D7C9485B7A6D2C3F1E018093B0E
:1016D4002A5E4F7D6CA5B48697E3F2C0D129380AFF
:1016E4001B6F7E4C5DB5A49687F3E2D0C139281AEE
:1016F4000B7F6E5C4DC6D7E5F48091A3B24A5B695B
:10170400780C1D2F3ED6C7F5E49081B3A25A4B79CD
:10171400681C0D3F2EE7F6C4D5A1B082936B7A48BE
:10172400592D3C0E1FF7E6D4C5B1A092837B6A58AD
:10173400493D2C1E0F7C2B2B2B7C0D6174680D7C7A
:1017440061747A0D004F4B0D0A0000000000000088
:101754000000000000000000004F4B0D0A000000D4
:1017640000000000000000000000000000434F4E95
:101774004E4543540D0A0000000000000000000024
:10178400004C495354454E0D0A000000000000006F
:1017940000000000004552524F520D0A00000000A4
:1017A400000000000000000000434F4E4E4543542B
:1017B400204641494C5552450D0A00000044495306
:1017C400434F4E4E45435445440D0A00000000006B
:1017D4000000000000000000000000000000000005
:1017E4000000000000FF13AFFF13B5FF13BAFF138F
:1017F400BEFF13C4FF13CAFF13CDFF13D2FF13D6CA
:10180400FF13DDFF13E0FF13E4FF13EBFF13F0FFFF
:0818140013F4FF13F8FF13FCAD
:0841D8007E137F84122FF522F3
:030023000223A411
:0B23A400C0E0C083C082C0D075D0181C
:1023AF002098030224F1C298750B01AF99300103F5
:1023BF0002247ABF020A906192E4F0D2010224F162
:1023CF002010030224F190175DE493B51F13906161
:1023DF00927401F09061957417F0A3745EF002246B
:1023EF0070901771E493B51F129061927402F09080
:1023FF0061957417F0A37472F08066901785E4935B
:10240F00B51F129061927403F09061957417F0A349
:10241F007486F0804C901799E493B51F12906192D7
:10242F007404F09061957417F0A3749AF080329051
:10243F0017ADE493B51F129061927405F0906195FA
:10244F007417F0A374AEF080189017C1E493B51F02
:10245F00109061927406F09061957417F0A374C296
:10246F00F0906192E0607BD2018077906192E0FE04
:10247F006040906195E0FCA3E0F5828C83E493B516
:10248F001F27906196E004F07006906195E004F0CC
:10249F00BF0A129061C7EEF0A3E4F0906192F0C210
:1024AF0001F52D803D052D8039906192E4F0C20138
:1024BF008030300B07C20B531F0F8017BF0904D298
:1024CF000B801FBF030D852D38632D80532D80C2C8
:1024DF0001800F7434252DF582E4346FF583EFF00E
:1024EF00052D2099030225B02002030225AE3009E5
:1024FF0079E534B4FF0B759902053475390002255F
:10250F00AEE534B52C147599030534906F33E07034
:10251F00030225AE7401F00225AEE534D3952C40AD
:10252F0006C202D2108078E53960133003064420CA
:10253F00F5998003853999053475390080617434B4
:10254F002534F582E43470F583E0F5396402600BCD
:10255F00E53964036005E539B40905759909803FCC
:10256F008539990534753900803574342534F582F1
:10257F00E43470F583E0FF7006C202D2108020C2EF
:10258F0010EFB47C090534750832C2028011AF34E4
:10259F00053474342FF582E43470F583E0F599C275
:0125AF009992
:0925B000D0D0D082D083D0E032FB
:10181C00C20ED20DC200907134741EF0E4907A990D
:10182C00F0C203C204C206C205F536C20AC20CC21B
:10183C0008906F33F090619774C4F0E4A3F0A37434
:10184C00C4F0A37401F0A374C8F0E4A3F0A374C8AB
:10185C00F0A37401F0A374C2F0E4A3F0A374C2F07B
:10186C00A37401F0E4A3F0A3F0F50F907BAFF0901C
:10187C007BAFE075F003A424E9F582E43417F5831B
:10188C00E493FB740193FA740293F9121C1770031E
:10189C00021C16E4907BB1F0A3F0907BB0F0907B2F
:1018AC00B0E024A6F582E43475F583E0FF70030202
:1018BC001C0D907BAFE075F003A424E9F582E434B1
:1018CC0017F583E493FB740193FA740293F9907BFC
:1018DC00B1E0F582758300121C30FEEFB5060F9057
:1018EC007BB27401F0907BB1E004F0021C04907B9D
:1018FC00B2E07003021C04EE6003021BFB907BAF92
:10190C00E0B410004003021C0D90191CF828287339
:10191C0002194C021999021C0D021C0D021AB0027C
:10192C001AE6021B15021AB5021B1A021B1F021B18
:10193C006D021B72021B77021BEB021BEF021BF3E7
:10194C00907BB0E024A6F9E43475FA7B01C0031B4C
:10195C008B59755A00755B00E4F55CD00312294C69
:10196C00907BB3121D60907BB3E0F8A3E0F9A3E089
:10197C00FAA3E0FB7F007E8C7D0A7C00121CAF1268
:10198C001D41907475EEF0A3EFF0021C0D907BB727
:10199C007461F0A37497F0907BB0E024A6F582E418
:1019AC003475F583E024D0F50FC394014007E50F9F
:1019BC00D394084003E4F50FE50F6028907BB7E45F
:1019CC0075F001121C5D85F082F58374C4F0150F5F
:1019DC00907BB7E475F001121C5D85F082F583E510
:1019EC000FF080D4907BB0E024A7F582E43475F539
:1019FC0083E024D0F50FC394014007E50FD394087E
:101A0C004003E4F50FE50F6028907BB7E475F00117
:101A1C00121C5D85F082F58374C8F0150F907BB7AE
:101A2C00E475F001121C5D85F082F583E50FF08002
:101A3C00D4907BB0E024A8F582E43475F583E024DF
:101A4C00D0F50FC394014007E50FD394084003E48D
:101A5C00F50FE50F6028907BB7E475F001121C5D63
:101A6C0085F082F58374C2F0150F907BB7E475F0A6
:101A7C0001121C5D85F082F583E50FF080D4907B1C
:101A8C00B7E475F001121C5D85F082F583E4F090EB
:101A9C007BB775F001121C5D85F082F583E4F0F5DF
:101AAC000F021C0DD208021C0D907BB0E024A6F98D
:101ABC00E43475FA7B01C0031B8B59755A00755BB6
:101ACC0000E4F55CD00312294C907BB3121D60909E
:101ADC007BB6E0907A99F0021C0D907BB0E024A6C6
:101AEC00F9E43475FA7B01C0031B8B59755A0075E8
:101AFC005B00E4F55CD00312294C907BB3121D60A3
:101B0C00907BB6E0F536021C0DD204021C0DD203FC
:101B1C00021C0D907BB0E024A6F9E43475FA7B012D
:101B2C00C0031B8B59755A00755B00E4F55CD00340
:101B3C0012294C907BB3121D60E4FFFEFDFC907BE0
:101B4C00B3E0F8A3E0F9A3E0FAA3E0FBD3121D4F36
:101B5C004008907BB6E0907134F0D20EC20D021C9E
:101B6C000DD206021C0DD200021C0DE4F50F907B69
:101B7C00B0E024A6F582E43475AF82907BB7F0A375
:101B8C00EFF0907BB7E0FEA3E0F5828E83E0FF647C
:101B9C0020602AEF6027E50FC394255020AE0F0577
:101BAC000F74022EF582E43461F583EFF0907BB86C
:101BBC00E004F07006907BB7E004F080C5AF0F0531
:101BCC000F74022FF582E43461F583740DF0740206
:101BDC00250FF582E43461F583E4F0F50F8022D211
:101BEC000A801ED20C801A906F337401F08012E4BC
:101BFC00907BB2F0907BB1F0907BB0E004F00218D7
:0A1C0C00AA907BAFE004F002187B01
:011C160022AB
:10344400E4F52A9061C8F0C207906193F0906F325E
:103454007405F0C202C210C201C20BE4F534F52CAB
:10346400F508F52DF50B90747574FFF0A374F4F062
:1034740012181C907134E004F528E4F53575F075E4
:10348400E535A42449F582E5F03468F583E4F0E5F4
:103494003575F00DA4242AF582E43461F583E4F053
:1034A400F52B75F068E535A42435F582E5F0347123
:1034B400F58375F00DE52B121D9DE4F0052BE52B2E
:1034C400B407DF0535E535B408B3E4F53DF525F576
:1034D40027F529F533F53CF52BF526F535F532F5C9
:1034E4009BC2ADF5C9D2CDD2CCC2C9C2CAF5CDF505
:1034F400CC907475E0F5CBA3E0F5CA85CBCD85CA35
:10350400CCD29ED29CD2CAC2ACC298C29975B81011
:0635140075B710D2AC22D5
:0100220022BB
:102DD4008F57300C0EE540B44209E543640270039A
:102DE400022EE8E54154E324DF605624DF60351405
:102DF400603224E36068147003022EAA1470030284
:102E04002ED124E2601E24606003022EE8E54275A0
:102E1400F00DA4242AF582E43461F5837D40AF5794
:102E24001228632275F00DE529A424F1F582E5F05A
:102E3400346BF5837D40AF57122863052953293F2E
:102E44002275F00DE525A424C9F582E5F03461F579
:102E5400837D40AF57122863052553257F2275F0E3
:102E640075E542A42456F582E5F03468F583E5431C
:102E7400543FFF1313543F75F00D121D9D7D40AF59
:102E84005712286375F068E542A42435F582E5F00D
:102E94003471F583E543543FFF1313543F75F00D2C
:102EA400121D9DE4F02275F068E542A42435F582F4
:102EB400E5F03471F583E543543FFF1313543F7534
:102EC400F00D121D9D7D40AF571228632275F075D9
:102ED400E542A42449F582E5F03468F5837D40AFEA
:052EE4005712286322D3
:10373E008F5A300307906002E04440F090600263BD
:10374E00A20190703463A201AF5A122875E4F52ECF
:10375E00F52F855A3190703463A20190153963A20A
:10376E0001AF31AE30AD2FAC2E1228A88F318E3076
:10377E008D2F8C2E7434255AF582E43470F583E542
:10378E002FF07435255AF582E43470F583E52EF06A
:10379E007434255AF582E43470F583E0F53AA3E0EB
:1037AE00F53BE55A2402F52C201B127E137FFD12E9
:1037BE002FF57E707F34E4FBAD2C1232967534FFFC
:0A37CE00D202C2992099FDD299227F
:10002600301122C211906F33E0600C04F0E0D394DB
:10003600F04004C2AF80FE906194E004F09061C885
:10004600E0600214F0E508B4010CE4F508D202C23F
:10005600992099FDD29930020F906194E0D39414BF
:10006600400BC202D2108005E4906194F090713486
:10007600E0FFE528D39F403C201B077E147F031238
:100086002FF5300E15E4906193F0C20DC209FF12F0
:1000960041719061C87402F08007E49061C8F0D2A3
:1000A60009E4F52DF538F52AF528C201906000F02F
:1000B600A3F0D2109061C7E0FF700302015024FE46
:1000C600601C14602514605114605A14606A24057B
:1000D6007078201B757E147F12122FF5806C201B02
:1000E600697E147F1D122FF58060201B077E147F0A
:1000F6002D122FF5300D53E4906193F0C20DC20915
:100106009061C8F0F52DF538752A03F528C20190DF
:100116006000F0A3F0D2108031201B2E7E147F3CAD
:10012600122FF58025201B077E147F4A122FF5908B
:100136007134E004F5288012201B077E147F6212BA
:100146002FF5907134E004F52822300D030202A742
:100156009061C8E060030202A72010030202A79084
:100166006193E014603114606E147003020250242F
:100176000360030202A27F01124171906193E004C1
:10018600F09061C87401F0301B030202A77E147F51
:1001960077122FF50202A7201B077E147F7C122FF1
:1001A600F578347C707D017BFF7A177939121E71E0
:1001B600E4F52DF538F5349061C7F00528C201D273
:1001C60002C2992099FDD299906193E004F0906162
:1001D600C8740AF00202A79061C7E0FFB403119049
:1001E60061937403F005289061C8743CF00202A77D
:1001F600EF6401601C201B0AEF70077E147F8812D3
:100206002FF59061C8740AF09061937401F00202B0
:10021600A7201B077E147F95122FF578347C707DFE
:10022600017B017A617902121E71E4F52DF538F52C
:1002360034C201D202C2992099FDD299906193E00D
:1002460004F09061C87406F080579061C7E0FFB46F
:100256000106A3743CF08049EFB4030A05289061B7
:10026600C8743CF0803BEFB40217E4F528D20DD2F7
:1002760009F52AC20F906000740BF0A374B8F080E1
:1002860020201B0AEF70077E147F88122FF59061DD
:10029600C8740AF09061937401F08005E49061934C
:1002A600F0E49061C7F0200D03020513E532C39414
:1002B600144003020513E5296527605A75F00DE51C
:1002C60027A424F5F582E5F0346BF583E02405F5E3
:1002D60057C3940E502E75F00DE527A424F1F58230
:1002E600E5F0346BF58363A20174042532F582E4EC
:1002F6003460F58363A201AF57122875E55725329E
:10030600F532800A201B077E147F9E122FF50527E3
:1003160053273F02051375F075E535A42449F58288
:10032600E5F03468F583E0700302042BE526705788
:1003360075F075E535A4244DF582E5F03468F5834E
:10034600E02405F557C3940E502E75F075E535A4D7
:100356002449F582E5F03468F58363A20174042527
:1003660032F582E43460F58363A201AF5712287533
:10037600E5572532F532800A201B077E147F9E1230
:100386002FF5052602051375F075E535A4244CF501
:1003960082E5F03468F583E0540FFFE526D39F50DD
:1003A6006775F075E535A4244DF582E5F03468F5FA
:1003B6008375F00DE526121D9DE02405F557C394BF
:1003C6000E503675F075E535A42449F582E5F0340E
:1003D60068F58375F00DE526121D9D63A201740470
:1003E6002532F582E43460F58363A201AF57122803
:1003F60075E5572532F532800A201B077E147F9E4D
:10040600122FF50526020513E4F52675F075E53578
:10041600A42449F582E5F03468F583E4F005355304
:1004260035070205130535533507E525653D605E3D
:10043600053D533D7F75F00DE53DA424CDF582E5E0
:10044600F03461F583E02405F557C3940E502F75FB
:10045600F00DE53DA424C9F582E5F03461F583632A
:10046600A20174042532F582E43460F58363A201A7
:10047600AF57122875E5572532F532020513301BA2
:10048600030205137E147F9E122FF5020513E53332
:1004960075F00DA4242AF582E43461F583E06068E2
:1004A600E53375F00DA4242EF582E43461F583E07E
:1004B6002405F557C3940E502DE53375F00DA4248D
:1004C6002AF582E43461F58363A20174042532F5CA
:1004D60082E43460F58363A201AF57122875E557AD
:1004E6002532F532800A201B077E147F9E122FF5D7
:1004F600E53375F00DA4242AF582E43461F583E42E
:10050600F0053353330780050533533307300203B1
:100516000205E7E50860030205E7200D030205E78B
:10052600E52A6401707B30072820082030030FE598
:1005360032600B200F089060027410F0801FE49068
:100546006002F0A37419F07F0212373EC20702055B
:10055600E7E5326028200F25E4906002F090600302
:100566007419F0E5322402FF12373E0528200802EE
:10057600D20FE4F532906000F0A3F08064D390606F
:1005860001E094E8906000E094034055E4F0A3F0A5
:10059600300F4EC20F201B497E147FA9122FF58003
:1005A60040E52A703C200406752A01F53222D390D4
:1005B6006001E094E8906000E094034024E4F0A336
:1005C600F0A374FEF0A374A0F0A374FFF07F0312EF
:1005D600373EE4F5320528201B077E147FB9122F1B
:1005E600F5E5387003020775F557E4F538F52EF58D
:1005F6002FE557547FF531E55754802434F582E4CE
:10060600346FF58363A20190153963A201AF31AE51
:1006160030AD2FAC2E1228A88F318E308D2F8C2E18
:10062600E55754802434F582E4346FAF82F5588F51
:100636005953577F74322557F582E4346FF583E0BA
:10064600FEA3E0653B7003EE653A7026201B077E2D
:10065600147FC4122FF5E52CB55711201B077E1405
:100666007FD8122FF574052528F52822740325282E
:10067600F528E52F452E6022301B030207757E14F0
:100686007FE2122FF5E4FBAD57AF59AE5812329602
:100696007D03AF2FAE2E1230DA22201B18E52A6416
:1006A6000160127E147FED122FF5E4FBAD57AF59B2
:1006B600AE58123296E557B40406E4F528C20F2266
:1006C600855982855883A3E024E760302499601F0A
:1006D60024F0600302076B752A01A2079207E4F56E
:1006E60032301B030207757E147FF2122FF522D2D9
:1006F60007201B7B7E147FFF122FF522E52A700B45
:10070600201B6C7E157F0C122FF522855982855889
:1007160083E030E405E4F528C20FD207E55724FC50
:10072600F551201B1A7E157F2C122FF5E559240250
:10073600FFE43558FEE55724FCFDE4FB123296E54E
:1007460051C3940F501BE5592402FFE43558F58335
:100756008F8263A201907A8563A201AF5112287538
:0F07660022E4F55122201B077E157F34122FF558
:010775002261
:1039A000020776E493A3F8E493A34003F68001F2C0
:1039B00008DFF48029E493A3F85407240CC8C33328
:1039C000C4540F4420C8834004F456800146F6DFF7
:1039D000E4800B01020408102040809041E0E47E66
:1039E000019360BCA3FF543F30E509541FFEE493EC
:1039F000A360010ECF54C025E060A840B8E493A3B3
:103A0000FAE493A3F8E493A3C8C582C8CAC583CADD
:103A1000F0A3C8C582C8CAC583CADFE9DEE780BE95
:0141E60000D8
:101C1700BB010689828A83E0225002E722BBFE02CB
:091C2700E32289828A83E49322FE
:101C3000BB010CE58229F582E5833AF583E0225069
:101C400006E92582F8E622BBFE06E92582F8E222B3
:0D1C5000E58229F582E5833AF583E49322CD
:101C5D00A3F8E0C5F025F0F0E5821582700215833A
:061C6D00E0C838F0E82297
:101C730075F008758200EF2FFFEE33FECD33CDCC28
:101C830033CCC58233C5829BED9AEC99E5829840AB
:101C93000CF582EE9BFEED9AFDEC99FC0FD5F0D688
:101CA300E4CEFBE4CDFAE4CCF9A88222B800C1B9B2
:101CB3000059BA002DEC8BF084CFCECDFCE5F0CBF0
:101CC300F97818EF2FFFEE33FEED33FDEC33FCEB29
:101CD30033FB10D703994004EB99FB0FD8E5E4F9E4
:101CE300FA227818EF2FFFEE33FEED33FDEC33FCD1
:101CF300C933C910D7059BE99A4007EC9BFCE99AC5
:101D0300F90FD8E0E4C9FAE4CCFB2275F010EF2F09
:101D1300FFEE33FEED33FDCC33CCC833C810D70709
:101D23009BEC9AE899400AED9BFDEC9AFCE899F844
:0E1D33000FD5F0DAE4CDFBE4CCFAE4C8F922D7
:0E1D4100C3E49FFFE49EFEE49DFDE49CFC22B3
:101D4F00EB9FF5F0EA9E42F0E99D42F0E89C45F0EA
:011D5F002261
:0C1D6000ECF0A3EDF0A3EEF0A3EFF022F6
:101D6C00A8828583F0D083D082121D83121D83122A
:101D7C001D83121D83E473E493A3C583C5F0C5834F
:101D8C00C8C582C8F0A3C583C5F0C583C8C582C8C1
:011D9C002224
:0C1D9D00A42582F582E5F03583F5832251
:10294C008B568A578958E4F562F561F560F55FF5A9
:10295C005DF55EE55A455B45596012EBC0E0EAC097
:10296C00E0E9C0E0AB59AA5AA95B121EDDAB5605D3
:10297C0058E558AA577002055714F9121C17F5633D
:10298C00C394094007E563D3940D40E1E5636420EB
:10299C0060DBE563B42D05435E038016E563B42B61
:1029AC0005435E01800C74FF2558F55874FF3557AC
:1029BC00F557E55C60046410703FAB56AA57A958F4
:1029CC00121C1764306009E55C702E755C0A802956
:1029DC00900001121C30FF64786004EFB45813436C
:1029EC005E01755C1074022558F558E43557F5579F
:1029FC008007E55C7003755C08AB560558E558AA72
:102A0C00577002055714F9121C17F563C3946140F3
:102A1C000AE563D3947A50035363DF74D02563F5CE
:102A2C0063C3940A400CE5639411406D74F92563FB
:102A3C00F563E563D3955C5060435E018562678501
:102A4C006166856065855F64AF5C7E00E4FCFDAB10
:102A5C0062AA61A960A85F121E8EC8ECC8C9EDC934
:102A6C00CAEECACBEFCBE4FCFDFEEB2563F562EEC0
:102A7C003AF561ED39F560EC38F55FAF62AE61ADFA
:102A8C0060FCAB67AA66A965A864D3121D4F5003FE
:102A9C00022A05435E04022A05E55E20E003E48079
:102AAC002DE55A455B4559601EAB56E55824FFF998
:102ABC00E55734FFFAEBC0E0EAC0E0E9C0E0AB59FF
:102ACC00AA5AA95B121EDDE55E30E20774FFFFFE19
:102ADC00FDFC22E55EAF62AE61AD60AC5F30E10340
:042AEC00021D412264
:101DA900E709F60870FA8046E709F20870FA803EFA
:101DB90088828C83E709F0A370FA807CE309F6082E
:101DC90070FA8074E309F20870FA806C88828C8357
:101DD900E309F0A370FA806089828A83E0A3F60898
:101DE90070FA805489828A83E0A3F20870FA8048E5
:101DF90080D280FA80C680D4806180F2802F8010E2
:101E090080A680EA809A80A880DA80E280CA802F42
:101E190089828A8363A20188828C8363A201E49305
:101E2900A363A201F0A363A20170F3800B89828AE4
:101E390083E493A3F60870F9ECFAA9F0EDFB228983
:101E4900828A8363A20188828C8363A201E0A363EF
:101E5900A201F0A363A20170F480DD89828A83E480
:101E690093A3F20870F980D088F0ED2402B404003D
:101E790050C6F582EB2402B4040050BC23234582EA
:051E890023901DF97318
:101E8E00E88FF0A4CC8BF0A42CFCE98EF0A42CFCF3
:101E9E008AF0EDA42CFCEA8EF0A4CDA8F08BF0A471
:101EAE002DCC3825F0FDE98FF0A42CCD35F0FCEBD0
:101EBE008EF0A4FEA9F0EB8FF0A4CFC5F02ECD3995
:0F1ECE00FEE43CFCEAA42DCE35F0FDE43CFC2202
:101EDD00BB011A89828A83D0F0D0E0F8D0E0F9D026
:101EED00E0FAD0E0FBE8C0E0C0F0021F355016E983
:101EFD00F8D083D082D0E0F9D0E0FAD0E0FBC082F8
:101F0D00C083021F2CBBFE16E9F8D083D082D0E02F
:0F1F1D00F9D0E0FAD0E0FBC082C083021F3E2261
:091F2C00EBF608EAF608E9F622DA
:091F3500EBF0A3EAF0A3E9F022AD
:091F3E00EBF208EAF208E9F222D4
:00000001FF
